:020000040000FA
:020000000528D1
:0800080009008316FF2390009C
:100010003E308500003095000030810083120030B2
:100020008B0007309900013085000130A3000301E7
:10003000E321C000F839031D2528F7216430A6000C
:10004000851929280122A60B2028B9010F30E921A2
:100050007F210130A5002508E321B90040302507A4
:10006000840039088000A50A10302506031D2B28BE
:10007000A2204019432841083106031D38284208B0
:100080003206031D382845306C21031D492877218D
:10009000702847306C21031D532883163C3085009F
:1000A00083128510702849306C21031D5D2883164A
:1000B0003A3085008312051170284B306C21031DE6
:1000C000672883162E3085008312051270284D3064
:1000D0006C21031D382883161E308500831285127B
:1000E0008C30A800A630A90085198228B120AA006A
:1000F0002A1882284008B0060319872802303006E3
:1001000003199728A90B7428A80B72289D28350875
:10011000B7003608B8000621AA002A189D2837081B
:100120003506031D982838083606031D98287028C0
:1001300083163E3085008312392883163E308500B1
:10014000831238288519A228B120AA002A18A228CB
:1001500040083006031DA2280621AA002A18A2285A
:1001600000340A30A600292285190134A60BB328D1
:100170005030A60085190029000000000000000092
:100180000000A60BBA28C830A6008519F528000083
:100190000000000000000000A60BC5280A30A600E1
:1001A000232285190134A60BD028FA30A600851920
:1001B000DF28000000000000A60BD728013406301D
:1001C000A6002322851D0134A60BE1281122851DDE
:1001D000F0281122851D01340130B0000B220034BB
:1001E0000330B00011220B2200340430A600232279
:1001F000851D0134A60BF7280230B00023220034FD
:100200001122851901340430B000003440191E2930
:100210002D212A1801343908B1002D212A18013462
:100220003908B20040181E292D212A180134390836
:10023000B3002D212A1801343908B4002D212A18C1
:1002400001343908B5002D213908B600401C0034AE
:100250003506AA00AA0F01340034A601B9012A14F8
:1002600040194F29F930A000851D3C2900000000ED
:100270000000A00B34290134C730A00085194329A0
:10028000A00B3E290134172240182922031085199A
:100290000314B90CA60AA61D3229AA01003417229C
:1002A0000310851D0314B90CA60AA6196729C730C7
:1002B000A00085195E29A00B59290134C730A00080
:1002C000851D6529A00B6029013429224F29851D30
:1002D00017221722AA010034840000083506031DE6
:1002E0000134840A00083606031D01340034A30BD0
:1002F0007D290230A3000510003405140034851D4B
:100300007F290530A6000510F7210514F721A60B5B
:10031000832985198929B120AA002A18892903303F
:100320003006031989293008C0000621AA002A18BE
:1003300089290130A5003030250784000008B90064
:100340002508E921A50A07302506031D9B29310848
:10035000C1003208C20005100430A7003508B700FC
:100360003608B800A22040083006031DB229401903
:10037000C12941083106031DB22942083206031D76
:10038000B22937083506031DC9293808360603196E
:10039000B2293508B9002508E921A50A3608B900AF
:1003A0002508E921A50A2708A6000514F72105104C
:1003B000F721A60BD529A70BAE294008B9000301E8
:1003C000E9210514003483169B001C141A088312BB
:1003D000080083169B0039089A001C1555309D00B3
:1003E000AA309D009C149C18F329831208006430E5
:1003F000A200F930A0000000A00BFB29A20BF929F4
:1004000000340A30A100F930A0000000A00B052A3A
:10041000A10B032A0034F930A0000000A00B0D2A24
:100420000034C730A0000000A00B132A0034953020
:10043000A0000000A00B192A00347C30A0000000AE
:10044000A00B1F2A00344A30A0000000A00B252A70
:1004500000343130A0000000A00B2B2A00341830EB
:0A046000A0000000A00B312A0034B8
:02400E00C43FAD
:00000001FF
